:100000000C9432040C94A8040C9418080C94A804C2
:100010000C94C8090C94A8040C94A8040C94A8048B
:100020000C94A8040C94A8040C94E81E0C94A80446
:100030000C944F2D0C94A8040C94A8040C94A804C0
:100040000C94A8040C94A8040C94A8040C94A80480
:100050000C94A8040C94A42D0C94A8040C94A8044B
:100060000C94A8040C94A8040C94A8040C94A80460
:100070000C94A8040C94A8040C94A8040C94A80450
:100080000C94A8040C94A8040C94A8040C94A80440
:100090000C94A8040C94A804490D570D630D630D2E
:1000A0003B0D630D630D630D630D630D630D630DF8
:1000B000630D630D630D630D630D630D3D0D630DE6
:1000C0003F0D630D630D630D630D5B0D630D720DCD
:1000D000590D630D630D630D630D630D630D630DAA
:1000E000630D630D630D630D630D630D330D4F0DD4
:1000F000410D530D630D430D630D470D630D510D00
:10010000450D550D4B0D4D0D630D630D630D630DC9
:10011000630D630D630D350D370D390D5D0D5F0DED
:10012000630D630D630D610D0F0E110E1B0E1B0E83
:100130001B0E1B0E1B0E1B0E130E150ED70D1B0ECA
:100140001B0E110E1E0E1B0E1B0ED70D0F0E1B0EBF
:100150001B0E150E1B0E1B0E1B0E1B0E1B0E1B0E5D
:10016000D90D0F0EFB0D1B0EFF0D1B0E1B0E1B0ED4
:10017000DB0D130E1B0E1B0E090E1B0E1B0E1B0E92
:10018000DD0D190E1B0EFD0D1B0E110E1B0E1B0E91
:100190000D0E010E1B0E030E150E1B0E1B0E1B0E5D
:1001A0000B0E050E1B0E1B0E1B0E1B0E1B0E1B0E2D
:1001B0001B0E070E1B0EDF0D1B0E1B0E130E1B0E50
:1001C0001B0E190E1B0E1B0E1B0E1B0E1B0E1B0EE9
:1001D0001B0E1B0E1B0EE10D1B0E1B0E1B0E090E24
:1001E0001B0E1B0E1B0E1B0E1B0E1B0E1B0E1B0EC7
:1001F0001B0E1B0EE30D1B0EE50DE70D1B0E1B0E5C
:100200001B0EE90DEB0DED0D1B0EEF0DF10D1B0E91
:100210001B0E1B0E170EF30D1B0EF70DF50DF90D32
:100220001B0E1B0E1B0E1B0E190E600EAE0E890E42
:10023000D40EFA0E020F090F0E0F120F2E103010EF
:100240003210341036103E103E103E1038103A1066
:100250003C1012112A113E1159116B1176119A118D
:10026000B311D911FB11E012851480166516331DE8
:100270005A1D521E5A1D521EA61DC91D521E201E59
:100280002F1E3C233C2374237423EF2323241A269C
:100290001A263A241A26CB23CB23D4251A26E9255D
:1002A0000726722530325820005220006973723AB6
:1002B0002530345820007725303258200021435310
:1002C000335F4630210A00214353335F5245414496
:1002D00059210A00214353335F5245534554210AA3
:1002E00000214353325F45305F4630210A002143ED
:1002F00053325F46302120253032580A00214353C3
:10030000325F4530210A00214353325F494E495440
:10031000210A00214353315F45305F253032582197
:100320000A00452575200050257520004D5B783A60
:10033000256420793A256420763A256420683A2598
:100340006420623A253032585D0A000A5B434C5201
:100350005D20004C257520000A4D6F7573653A20AD
:1003600025730A000A4445463A20000A4558503A87
:1003700020000A494E543A20000A4C4F473A2000C8
:100380000A4C4D533A200053257520000A49443A3F
:100390002530345828257325732920000A556E6BA3
:1003A0006E6F776E2049443A205265706F727420E8
:1003B000746F20544D4B20004E4720004F4B2000BF
:1003C0004E4720004F4B20000A353537365F4353E8
:1003D0003832683A0052257520005725752000579D
:1003E00025752000572575200058257520004125CA
:1003F00075200049257520005B4348475D20000AB1
:100400002575205052543A25303258204953523ADB
:100410002530345820000A2575204552523A25309F
:100420003258204953523A253034582000535B2526
:10043000303258202530325820253032585D200087
:10044000007B46010203763A687F6577482B353B8F
:100450006978796439141E3C6A7A1D16041A1F3DA6
:100460006B061B070821203E6C2C19091715223F2B
:100470006D11050B0A1C23406E7E100D18242541BA
:100480006F360E0C122726427037380F33132D4368
:10049000717534322F2E44727C7D2830317445734F
:1004A00051504A524D492A5466594F5C5F4C4B4E4D
:1004B00062635A5D5E60295367585B5657614755C2
:1004C0004842403E3C3A3B456843413F3D2B357EE8
:1004D000697A790078141E7B6A7C1D16041A1F7FC6
:1004E0006B061B07082120656C2C19091715224A79
:1004F0006D11050B0A1C234C6E49100D1824255153
:100500006F360E0C1227264F7037380F33132D52CB
:10051000717534502F2E4E72397D28304D314B730A
:100520005464586776012A773259745C5F66020317
:1005300062635A5D5E60295344575B565561474676
:1005400080291E1F20212223242526272D2E2A2BF9
:10055000141A0815171C180C12132F3028780416BB
:1005600007090A0B0D0E0F33343579311D1B06199F
:100570000511103637387D557A2C393A3B3C3D3ED3
:100580003F4041424353475F6061565C5D5E57594F
:100590005A5B62634648644445677B7F650301029A
:1005A0005250514F68696A6B6C6D6E6F7071725802
:1005B00000494C754A4D734B4E767C777E74665479
:1005C0000A4C6F6F702073746172742E0A000A55A2
:1005D000534220636F6E666967757265642E0A0008
:1005E0000A544D4B3A6137373931342F4C55464117
:1005F0003A6436613764660A003403490042004DAC
:100600000020005000430020006B0065007900626C
:10061000006F00610072006400200063006F006ED4
:10062000007600650072007400650072000000082A
:100630000354004D004B0000000403090409025458
:1006400000030100A03209040000010301010009B8
:100650002111010001223900070581032000010951
:100660000401000103010200092111010001227FA0
:1006700000070582030800010904020001030000CD
:100680000009211101000122220007058303200037
:10069000011201100100000008EDFEEE1B01020135
:1006A0000200010631FF0974A1010975150026FF3A
:1006B000009520750881020976150026FF00952017
:1006C00075089102C005010902A1010901A1008577
:1006D00001050919012908150025019508750181F1
:1006E000020501093009311581257F9502750881C0
:1006F0000609381581257F950175088106050C0AC4
:1007000038021581257F950175088106C0C0050155
:100710000980A10185021601002637001A81002AEE
:10072000B700751095018100C0050C0901A1018574
:1007300003160100269C021A01002A9C02751095DE
:10074000018100C005010906A101050719E029E79B
:100750001500250195087501810205081901290573
:100760009505750191029501750391010507190021
:1007700029F71500250195F875018102C0636F6E98
:1007800073756D65723A20253034580A0073797399
:1007900074656D3A20253034580A000A002530323D
:1007A0005820006B6579626F6172643A20004C4595
:1007B000443A20253032580A0025583A253031363F
:1007C0006225730A000A202030313233343536373F
:1007D00038394142434445460A0064656C5F6B65A5
:1007E000795F6269743A2063616E27742064656C76
:1007F0003A20253032580A006164645F6B65795F86
:100800006269743A2063616E2774206164643A20DF
:10081000253032580A00290A002575002F00257559
:10082000005D280025640020002564002000256468
:100830000020002564007C0025303258006D6F7563
:1008400073656B6579205B62746E7C7820792076A5
:1008500020685D287265702F61636C293A205B0007
:10086000780B0F1711241FBECFEFD0E2DEBFCDBF34
:1008700004B603FE49C08091210490912204A09106
:100880002304B09124048730904BA740B04B09F06B
:100890003BC0109221041092220410922304109263
:1008A000240414BE0FB6F894A89580916000886166
:1008B00080936000109260000FBE109201081092A9
:1008C0000008E3E0F0E089E080935700E491E695CA
:1008D000E370E150E33040F4F0E0EE0FFF1FE85822
:1008E000FE4F2081318102C020E030E280E090E0C4
:1008F000A2E0B0E0821B930BA109B109B595A795C1
:1009000097958795FC01099511E0A0E0B1E0ECEF27
:10091000F3E600E00BBF02C007900D92AE37B107BF
:10092000D9F724E0AEE7B1E001C01D92A132B207D1
:10093000E1F714E0C2E3D4E004C02197FE010E9475
:10094000DF31C033D107C9F70E944C1A0C94FC3137
:100950000C940000FF93EF93E0917E01F0917F01F2
:10096000309709F00995EF91FF910895FC01859169
:10097000803011F0EFDFFBCF0895FF27E0E230E297
:1009800047FF0CC0419597FF09C0EDE26095709557
:1009900080959095611D711D811D911D27FF02C0DD
:1009A000219530E350E2AA27660F771F881F991F11
:1009B000AA1FA41710F0A41B63955A95A9F7AA3093
:1009C00008F0A95FA05DAF93F395611571058105EE
:1009D000910541F7ED3211F4EF93F395F21718F406
:1009E0003F93F395FBCF8F91B5DFFA95E1F708952B
:1009F000E991F9918591803021F0853219F0AADFD3
:100A0000F9CF089520E0E89455915532C1F3503361
:100A100011F4689455915A3348F4505390F3220FCF
:100A2000022E220F220F200D250FF4CF0EF4219558
:100A300089919991533619F3533729F1533559F167
:100A4000BC0188279927E8945C3621F48991999113
:100A500068945591543639F446EF7EF077FF0DC017
:100A60008FEF9FEF0AC055374AE039F0583540E123
:100A700021F0523642E009F00895FF93EF937DDFB5
:100A8000EF91FF91B7CFFF93EF93FC0181918030FD
:100A9000B9F360DFFBCFFF93EF9368DFF1CFDF9314
:100AA000CF93CDB7DEB72596A3DFCF91DF91089521
:100AB000FC012AB1938D909592239AB99BB1838DB5
:100AC000892B8BB90895FC019AB1838D8095892378
:100AD0008AB99BB1838D892B8BB985E08A95F1F713
:100AE000000099B1838D982381E009F480E0089596
:100AF000FC012BB1948D909592239BB99AB1848D72
:100B0000892B8AB90895FC012AB1948D909592237E
:100B10009AB99BB1848D892B8BB90895FC019AB148
:100B2000848D809589238AB99BB1848D892B8BB95B
:100B300085E08A95F1F7000099B1848D982381E0D2
:100B400009F480E008950F931F93CF93DF938C01F6
:100B5000EB01C8010E946305882341F0209731F022
:100B600085E08A95F1F700002197F3CFCE01DF9160
:100B7000CF911F910F9108950F931F93CF93DF9300
:100B80008C01EB01C8010E946305811108C0209708
:100B900031F085E08A95F1F700002197F3CFCE017F
:100BA000DF91CF911F910F910895CF93DF93EC01C7
:100BB0000E945805CE01DF91CF910C9483053BB183
:100BC000FC01238D209523232BB93AB1238D232BB0
:100BD0002AB90C948305FC018CB3938D982B9CBB94
:100BE0009DB3838D892B8DBB0895CF93DF93EC014B
:100BF0000E94EB05CE01DF91CF910C94D505FC014D
:100C00002DB3938D909592239DBBCF010C94DF055E
:100C1000FC01118210821282138280E090E8958399
:100C20008483178210860895CF93DF93EC012E986A
:100C300026982F9827980E94DF05898D843080F4AC
:100C400040916900880F22E030E0B90102C0660FD0
:100C5000771F8A95E2F7CB01842B8093690010C03F
:100C600040916A008370880F22E030E0B90102C031
:100C7000660F771F8A95E2F7CB01842B80936A0079
:100C80009DB38B8D809589238DBBCE01DF91CF9154
:100C90000C940806CF93DF93EC018F8190E00196CE
:100CA0008F709927288530E08217930749F4CE0189
:100CB0000E940806CE010E94EB05CE010E94D505D8
:100CC0002FB7F89498858F81891751F0FE01E90FAD
:100CD000F11D81859F5F9F709887C82FD0E002C06B
:100CE000CFEFDFEF2FBFCF3F8FEFD80781F080919D
:100CF000060480FF0CC0DF93CF9382EA92E09F93BB
:100D00008F930E944F050F900F900F900F90CE0180
:100D1000DF91CF9108950F931F93CF938C01CAE178
:100D2000C15071F0C8010E944A068F3F2FEF920711
:100D300049F48FE99FE00197F1F700C00000F0CF80
:100D40008FEF9FEFCF911F910F9108952F923F92B8
:100D50004F925F926F927F928F929F92AF92BF92CB
:100D6000CF92DF92EF92FF920F931F93CF93DF9377
:100D7000EC01062F1B828091060480FF0CC01F929D
:100D80006F9386EB92E09F938F930E944F050F9095
:100D90000F900F900F908C819D818115904899F054
:100DA0008091060480FF19C18C819D819F938F9350
:100DB0008CEA92E09F938F930E944F050F900F90C3
:100DC0000F900F900AC19DB38B8D809589238DBBA9
:100DD0002BE0A22EBB24B39410E09924939438E026
:100DE000232E47E0342E56E0452E65E0562E74E063
:100DF000872EE3E07E2EF2E06F2EA9EACA2EA2E053
:100E0000DA2ECE010E94DF058FE193E00197F1F722
:100E100000C00000CE010E9478058FE193E00197A9
:100E2000F1F700C00000CE010E94580568E97AE39E
:100E3000CE010E94A305892B11F49B826FC0E12C87
:100E4000F12C90E59A95F1F7C8010E2C02C095950A
:100E500087950A94E2F780FF05C0B924CE010E946D
:100E6000830503C0CE010E94780562E370E0CE01E5
:100E70000E94BC05892B11F46B8250C062E370E0C4
:100E8000CE010E94A305892B11F47B8247C02FEF6E
:100E9000E21AF20A88E0E816F10499F690E59A95CC
:100EA000F1F7CE01BB2019F00E94830502C00E9419
:100EB000780562E370E0CE010E94BC05892B11F435
:100EC0008B822CC062E370E0CE010E94A305892BC7
:100ED00011F45B8223C020E52A95F1F7CE010E9430
:100EE00083059CE2E92EFF24F394CE010E948E0537
:100EF000882329F0E114F104C9F44B820FC0EF28D4
:100F0000E1F38CE2E82EFF24F394CE010E948E05DB
:100F1000811114C0E114F104D1F53B828B81813041
:100F200009F049C0AA94A1103AC045C085E08A954D
:100F3000F1F7000091E0E91AF108D7CFEF2869F343
:100F40006CE271E0CE010E94BC05892B11F42B826A
:100F5000E5CFCE010E940806CE010E94D505CE0144
:100F60000E94EB05CE01DF91CF911F910F91FF9071
:100F7000EF90DF90CF90BF90AF909F908F907F9039
:100F80006F905F904F903F902F900C948B0625E0D0
:100F90002A95F1F7000081E0E81AF108B6CF1B822C
:100FA0008091060480FF2DCFDF92CF920E944F05E3
:100FB0000F900F9026CF8B8180618B83CE010E9492
:100FC000DF058FE39FE10197F1F700C00000CE013C
:100FD0000E94D505CE010E94EB058FEF9FEFDF91B8
:100FE000CF911F910F91FF90EF90DF90CF90BF9026
:100FF000AF909F908F907F906F905F904F903F90B9
:101000002F9008951F93CF93DF93EC01162F6DEE71
:101010000E94A6068A3F910539F4612FCE01DF9127
:10102000CF911F910C94A606DF91CF911F91089547
:101030001F920F920FB60F9211240BB60F922F939F
:101040003F934F935F938F939F93EF93FF9349B198
:101050005091B701909107042091A1013091A20114
:101060002115304819F49093A3010FC08091A3017A
:10107000981B933050F08091A1019091A201909320
:101080009E0180939D0180E21AC12091A1013091BF
:10109000A201369527953093A2012093A10181E00A
:1010A00090E001C0880F5A95EAF7842349F08091B7
:1010B000A1019091A20190689093A2018093A10157
:1010C0008091A1019091A20199278038910509F49E
:1010D00050C1A8F48032910509F44BC138F400974F
:1010E00009F447C1409709F495C0DEC080349105EA
:1010F00009F43FC18035910509F48CC0D5C0803C0E
:10110000910531F148F48039910509F483C0803AA2
:10111000910509F44DC0C8C0803D910509F47AC01D
:10112000803E910509F0C0C08091A1019091A2017B
:1011300090939E0180939D018091A1019091A201C5
:10114000892F99279093A2018093A10183E256C031
:1011500080919F01811123C084E629B19091B8014B
:10116000922311F48111EDC029B19091B80192231D
:10117000E1F08111ECC08091A1019091A2019093C6
:101180009E0180939D018091A1019091A201892FE0
:1011900099279093A2018093A10182E22FC08091B0
:1011A0009F01823209F0E5C0E6CF8111E2C0E3CFB2
:1011B00080919F01811125C084E629B19091B801E9
:1011C000922311F48111C9C029B19091B8019223E1
:1011D000F1F08111C8C08091A1019091A20190937A
:1011E0009E0180939D018091A1019091A201892F80
:1011F00099279093A2018093A10181E280939F019E
:101200006BC080919F01813209F0B3C0E4CF81119E
:10121000B0C0E1CF8091A1019091A20190939E0175
:1012200080939D018091A1019091A20180399A4AF9
:1012300011F482E044C02091A1013091A20180917B
:10124000A1019091A20124E0329F212D3327112486
:10125000217056E0969587955A95E1F78227982F49
:101260009E7F29F0982F969581708927F8CF81115C
:1012700002C081E024C08091A1019091A20197FF5A
:1012800002C080E101C081E180939F018091A101B2
:101290009091A20126E0969587952A95E1F7909383
:1012A000A2018093A10118C010929F018091A10119
:1012B0009091A20190939E0180939D0180E880937C
:1012C000A0019BB18091B801282F209592239BB952
:1012D0009AB1892B8AB92EC02091A1013091A20127
:1012E0008091A401E82FF0E0E356FE4F21878F5F45
:1012F0008F708093A40190E001968F7099273091B0
:10130000A501432F50E08417950769F42DB3809110
:10131000B801482F409524232DBB9BB194239BB942
:101320009AB1892B8AB98091A401831303C080E408
:101330008093A00180E090E89093A2018093A101A6
:1013400018C095E09A95F1F70000815006CF25E08E
:101350002A95F1F70000815007CF95E09A95F1F7B3
:10136000000081502ACF25E02A95F1F70000815036
:101370002BCFFF91EF919F918F915F914F913F9173
:101380002F910F900BBE0F900FBE0F901F901895CE
:101390001F920F920FB60F9211240BB60F922F933C
:1013A0003F934F935F938F939F93EF93FF9349B135
:1013B00050919A0190910704209184013091850108
:1013C0002115304819F4909386010FC08091860151
:1013D000981B933050F080918401909185019093F7
:1013E00081018093800180E21AC1209184013091B3
:1013F000850136952795309385012093840181E0FE
:1014000090E001C0880F5A95EAF7842349F0809153
:101410008401909185019068909385018093840167
:10142000809184019091850199278038910509F474
:1014300050C1A8F48032910509F44BC138F40097EB
:1014400009F447C1409709F495C0DEC08034910586
:1014500009F43FC18035910509F48CC0D5C0803CAA
:10146000910531F148F48039910509F483C0803A3F
:10147000910509F44DC0C8C0803D910509F47AC0BA
:10148000803E910509F0C0C0809184019091850152
:1014900090938101809380018091840190918501D6
:1014A000892F9927909385018093840183E256C008
:1014B00080918201811123C084E629B190919B0122
:1014C000922311F48111EDC029B190919B019223D7
:1014D000E1F08111ECC0809184019091850190939D
:1014E0008101809380018091840190918501892FF1
:1014F0009927909385018093840182E22FC0809187
:101500008201823209F0E5C0E6CF8111E2C0E3CF6B
:1015100080918201811125C084E629B190919B01BF
:10152000922311F48111C9C029B190919B0192239A
:10153000F1F08111C8C08091840190918501909350
:101540008101809380018091840190918501892F90
:101550009927909385018093840181E28093820191
:101560006BC080918201813209F0B3C0E4CF811158
:10157000B0C0E1CF80918401909185019093810169
:1015800080938001809184019091850180399A4AED
:1015900011F482E044C02091840130918501809152
:1015A00084019091850124E0329F212D332711245D
:1015B000217056E0969587955A95E1F78227982FE6
:1015C0009E7F29F0982F969581708927F8CF8111F9
:1015D00002C081E024C0809184019091850197FF31
:1015E00002C080E101C081E1809382018091840189
:1015F0009091850126E0969587952A95E1F790933D
:1016000085018093840118C0109282018091840129
:1016100090918501909381018093800180E880936F
:1016200083019BB180919B01282F209592239BB928
:101630009AB1892B8AB92EC02091840130918501FD
:1016400080918701E82FF0E0E058FE4F21878F5FFF
:101650008F708093870190E001968F709927309169
:101660008801432F50E08417950769F42DB38091CA
:101670009B01482F409524232DBB9BB194239BB9FC
:101680009AB1892B8AB980918701831303C080E4C2
:101690008093830180E090E890938501809384019A
:1016A00018C095E09A95F1F70000815006CF25E02B
:1016B0002A95F1F70000815007CF95E09A95F1F750
:1016C000000081502ACF25E02A95F1F700008150D3
:1016D0002BCFFF91EF919F918F915F914F913F9110
:1016E0002F910F900BBE0F900FBE0F901F9018956B
:1016F000EDE9F1E0118210821282138220E030E8DD
:1017000035832483168291E0918F128E82E0838F3D
:10171000948FE0E8F1E01182108212821382358307
:101720002483168293E0918F828F88E0838F84E0F8
:10173000848F0895262F30E094E0359527959A956B
:10174000E1F72770E62FEF70823069F08330A1F067
:101750008130E1F4F0E080E1289FE00DF11D1124DB
:10176000E05CFA4F11C0F0E080E1289FE00DF11D30
:101770001124E054FB4F08C0F0E080E1289FE00D09
:10178000F11D1124E05CFB4F8491089580E80895D9
:101790000F931F93CF93DF938C01EB0169EEFC0154
:1017A000808191810E94A606F801808191810E942A
:1017B0008B068883F801808191810E948B06898342
:1017C000F801808191810E948B068A8399279F93DB
:1017D0008F9389811F928F9388811F928F938DE2BF
:1017E00094E09F938F930E944F058DB79EB7089604
:1017F0000FB6F8949EBF0FBE8DBFDF91CF911F91A2
:101800000F910895E6EDF1E01192119281E0E63E2C
:10181000F807D1F70895CF93DF93EC011B821A826A
:101820001C821D820E94020C88819981DF91CF91D8
:101830000C9414061F93CF93DF93FC0184810E94C4
:101840009A0B87FD20C0182F1F70C82FD0E094E09E
:10185000D595C7959A95E1F7612F8C2F0E94562157
:10186000811111C0CC0FDD1FCA52DE4F81E090E024
:1018700002C0880F991F1A95E2F728813981822BBF
:10188000932B99838883DF91CF911F9108951F93A4
:10189000CF93DF93FC0184810E949A0B87FD22C0C5
:1018A000182F1F70C82FD0E094E0D595C7959A9552
:1018B000E1F7612F8C2F0E945621882399F0CC0FDD
:1018C000DD1FCA52DE4F81E090E002C0880F991FF1
:1018D0001A95E2F780959095288139818223932388
:1018E00099838883DF91CF911F91089588EC91E0CF
:1018F0000E940B0C8AEB91E00C940B0C8091060477
:101900008160809306040C94020CE82FF0E0EE0F47
:10191000FF1FEA52FE4F8081918108950C94020CC2
:101920007770E72FF0E098E0899FE00DF11D11241A
:1019300084E0EE0FFF1F8A95E1F76F70E60FF11D4F
:10194000EE0FFF1FE050F849859194910895FC0136
:101950008481823070F0843061F062FB992790F9C5
:1019600060FD926061FD9460692F808191810C948B
:1019700002080895CF93C82F682F88EC91E00E9449
:10198000A70C6C2F8AEB91E0CF910C94A70CCF920F
:10199000DF92EF92FF920F931F93CF93DF936C012F
:1019A0008B010E947D2D7C01F601808191810E9436
:1019B0004A06EC01019631F4C7010E94952D80176B
:1019C000910790F3CE01DF91CF911F910F91FF907E
:1019D000EF90DF90CF9008950F931F93CF93DF93F5
:1019E000FC0180819181DC0112962C912131F9F06A
:1019F0008F0162EF0E94A6068F3FBFEF9B07D1F0D9
:101A00008A3F9105D1F464EF71E0C8010E94C70CD0
:101A10008F3F2FEF9207A1F0D82FCC2764EF71E012
:101A2000C8010E94C70CDE01A82BCD010BC08DEFB1
:101A30009FEF08C08FEF9FEF05C08EEF9FEF02C0B2
:101A400080E090E0DF91CF911F910F910895CF93A7
:101A5000862F90E0FC017C97E834F105A0F5E45B6B
:101A6000FF4F0C94DF3185E53EC08AE53CC08BE535
:101A70003AC08CE538C08DE536C08EE534C08FE5C0
:101A800032C080E630C081E62EC082E62CC083E6FC
:101A90002AC08FE628C081E726C082E724C084E7F9
:101AA00022C085E720C087E71EC088E71CC08AE700
:101AB0001AC08CE718C08FE716C080E714C089E70A
:101AC00012C08BE710C0C62F1F926F9383E193E083
:101AD0009F938F930E944F050F900F900F900F9040
:101AE0008C2F01C084E5CF910895CF93DF93EC0153
:101AF00099859230A9F128F4992341F09130C9F0E9
:101B000045C09330B1F19430D9F140C0603E21F02E
:101B1000613E21F482E02BC081E029C067FD04C052
:101B2000CE010E941A0C33C06F77CE010E94470C81
:101B30002EC0663359F118F46A3229F427C06A3A84
:101B400029F1663B19F167FD05C0CE010E94270D02
:101B5000682F12C06F77CE010E94270D682F13C027
:101B60006D3121F06D3991F484E001C083E0898703
:101B70000EC0653459F465E5CE010E941A0C06C00A
:101B8000653C21F465E5CE010E94470C198680E092
:101B9000DF91CF910895862F90E0FC013397E138D3
:101BA000F10508F048C0EC56FF4F0C94DF3189E195
:101BB000089587E108958FE1089587E2089580E60A
:101BC000089582E608958CE5089583E508958FE2EF
:101BD000089589E3089587E308958FE3089587E4DE
:101BE00008958FE4089586E508958EE508958FE7BA
:101BF000089580E0089585E608958EE608958FE6BD
:101C0000089580E3089588E3089580E4089588E4C2
:101C1000089580E5089587E508958FE5089588E1A2
:101C2000089588E0089580E2089580E108958DE6A2
:101C3000089588E20895862F8F7708958FE008959C
:101C40006B35C9F068F46131F1F020F46E30C9F4FD
:101C500084E50895633169F0643599F48BE508955E
:101C60006D3559F050F0623651F06C3751F487E71A
:101C7000089581E108958DE508958AE608958EE03E
:101C80000895862F08958FE00895613131F0613411
:101C900011F48CE70895862F089583E108951F932A
:101CA000CF93DF93EC01162FEA858E2F90E08930D9
:101CB000910508F0BDC0FC01EB5EFE4F0C94DF31D6
:101CC0008A819B8180599B4A029720F4CE010E9411
:101CD000200E182F103E69F030F4133871F01438CC
:101CE00071F46FE792C0113E31F0103F41F481E092
:101CF00093C082E091C084E08FC062E086C01A8603
:101D000017FD02C0612F21C00E94020C87E093E002
:101D100069C08A819B8180599B4A029720F4CE0139
:101D20000E94450E182F193509F482C0103F19F092
:101D3000123119F47DC083E06FC01A8617FD09C007
:101D4000612FCE010E94CB0D682FCE010E941A0C8C
:101D500070C00E94020C8DEF92E044C08A819B818A
:101D600080599B4A029720F4CE010E94200E182F22
:101D7000133821F0143821F46FE757C062E055C0E2
:101D80001A8617FD02C0612F25C00E94020C1F9207
:101D90001F938EEE92E09F938F930E944F050F90BA
:101DA0000F900F900F9024C08A819B8180599B4A8D
:101DB000029720F4CE010E94450E182F1A86123188
:101DC000C1F11935B1F117FD09C0612FCE010E9493
:101DD000CB0D682FCE010E94470C2BC00E94020C35
:101DE00081EE92E09F938F930E944F050F900F908A
:101DF0008FEF20C0643121F0603FD1F486E00CC049
:101E000085E00AC06737A1F460E0CE010E941A0C99
:101E10000FC0643169F487E08A870BC0603F41F4EA
:101E200088E0FACF673721F460E0CE010E94470CCA
:101E30001A8680E0DF91CF911F9108956C3551F0A3
:101E400018F4633169F00AC0663731F06E3731F447
:101E500086E7089581E508958EE70895862F089511
:101E60008DE50895663809F466C058F5673609F4BB
:101E700050C0A0F46C3509F464C040F4683009F433
:101E800064C0673509F05FC08CE50895643609F4D5
:101E900044C0653609F057C08DE60895673709F4E8
:101EA0004EC038F46D36B9F16E3609F04CC085E697
:101EB00008956438A1F1E8F56C3709F044C088E66C
:101EC00008956C38A1F178F4693869F130F4673815
:101ED00041F16838C1F58EE708956A3831F16B3801
:101EE00091F584E008956F3881F030F46D3859F041
:101EF0006E3849F587E608956139F9F040F06239A6
:101F000011F589E0089587E708958FE708958BE735
:101F1000089582E6089584E608958EE608958CE794
:101F2000089582E008958CE0089583E0089585E0A7
:101F3000089588E0089580E1089581E0089588E596
:101F4000089583E50895862F089586E70895CF9331
:101F5000DF93EC016F3B41F028F486E5860F823079
:101F600070F402C06C3F59F41B8684ED92E09F939D
:101F70008F930E944F050F900F908FEFC1C08B85FC
:101F8000813009F44DC038F0823009F486C08330C6
:101F900009F4A1C0B4C08A819B8182392BEA9207DF
:101FA00021F4CE010E941E0F06C081399B4A21F404
:101FB000CE010E94320F682F663809F168F4633849
:101FC000D1F020F4603819F582E07FC06438A9F0C0
:101FD0006538E9F468E61DC06C38A9F030F467385C
:101FE00081F06B38A1F461E014C06D3871F0603F8E
:101FF00071F481E06AC062E00CC06FE70AC068E774
:1020000008C060E006C069E004C06AE002C067FD85
:1020100004C0CE010E941A0C72C087EC92E036C058
:102020001B868A819B8182392BEA920721F4CE019B
:102030000E941E0F06C081399B4A21F4CE010E94E6
:10204000320F682F862F90E0FC01E358F109EB3046
:10205000F105A0F4E25EFE4F0C94DF3162E010C0A7
:102060006FE70EC068E60CC068E70AC060E008C011
:1020700061E006C069E004C06AE002C067FD04C018
:10208000CE010E94470C3BC08DEB92E09F938F9353
:102090000E944F050F900F9032C0653279F030F4F6
:1020A000663171F06E3199F460E00BC0663221F058
:1020B000603F69F483E009C06DE503C063E501C0DA
:1020C00061E5CE010E941A0C04C08B8718C00E94E3
:1020D000020C1B8614C06E3169F020F46631B9F72A
:1020E00061E509C0653221F0663289F76DE503C00C
:1020F00063E501C060E0CE010E94470CEACF80E0BA
:10210000DF91CF9108958F929F92AF92BF92CF921D
:10211000DF92EF92FF920F931F93CF93DF9300D044
:1021200000D01F92CDB7DEB78C01DC01ED91FC91A0
:102130008381882391F1E080F180D3800E947D2DFE
:10214000FF92EF921F92DF929F938F9386E194E02C
:102150009F938F930E944F05D801ED91FC911197A9
:10216000838180750FB6F894DEBF0FBECDBF79F4C2
:1021700018968C9118978B3019F48CE018968C93E4
:102180008381823021F48DE0D80118968C931382DC
:10219000D801ED91FC9111821082D801ED91FC9152
:1021A00011978281882381F1928115968C919817DD
:1021B00059F1E080F180D2800E947D2DFF92EF9254
:1021C0001F92DF929F938F938FEF93E09F938F9354
:1021D0000E944F05F80185810FB6F894DEBF0FBE4F
:1021E000CDBF0190F081E02D85FF03C0928194FD69
:1021F0009FC584FD9AC5D801ED91FC91119782810C
:1022000015968C9311821082D8011896EC918E2F1E
:1022100090E08E30910508F0E7C5FC01E75DFE4FC8
:102220000C94DF310E947D2D9F938F9383EF93E079
:102230009F938F930E944F050E947D2DF8019783F5
:102240008683808191810E94F50581E0D8011896EE
:102250008C936BC0F801808191810E944A0601969F
:10226000C9F7D80116968D919C9117970E94952DCC
:10227000893B9B4008F4B8C582E03FC50E947D2D94
:102280009F938F938EEE93E09F938F930E944F05C1
:102290006FEFD8018D919C910E94A6060F900F9030
:1022A0000F900F908A3F910511F486E026C583E0D8
:1022B0006FC3F801808191810E94FF052E98269AB4
:1022C0002F98279A0E947D2DD80117969C938E9364
:1022D000169784E05EC3F801868197810E94952D50
:1022E000853F914008F480C585E052C32E9826981A
:1022F0002F982798F801808191810E940806D801C3
:102300008D919C910E94F5050E947D2D9F938F9346
:1023100089EE93E09F938F930E944F050E947D2D3D
:10232000F8019783868386E080870F900F900F9047
:102330000F905AC5D8018D919C910E944A06019632
:1023400009F452C50E947D2D9F938F9384EE93E0F4
:102350009F938F930E944F050E947D2DF8019783D4
:10236000868387E0E1CFD80116968D919C911797CF
:102370000E94952D853F914018F089E0F8018087F3
:10238000D8018D919C910E944A06019609F42CC5B2
:102390000E947D2D9F938F938FED93E09F938F935A
:1023A0000E944F050E947D2DF8019783868388E067
:1023B000BBCFD80116968D919C9117970E94952DB1
:1023C000853F914018F089E0F8018087D8018D9110
:1023D0009C910E944A06019609F406C50E947D2D33
:1023E0009F938F938AED93E09F938F930E944F0565
:1023F00089E0F80199CFC8010E94EC0CD80113962E
:102400009C938E9312970E947D2D9F938F9385EDC1
:1024100093E09F938F930E944F05F80182819381EF
:102420000F900F900F900F90009711F482E010C062
:102430008F3FBFEF9B0711F481E044C09C012D5FEB
:102440003F4F2230310590F38F3F910529F484E00E
:10245000D80114968C9372C09C0125583B4A2230B7
:10246000310508F49DC48239BBEA9B0709F498C47E
:102470009C0120593B4A22303105F8F488EC93E066
:102480009F938F930E944F0582E0F801848360EF51
:10249000808191810E94A6060F900F908A3F91053E
:1024A000F1F562E8D8018D919C910E94A6068A3FC1
:1024B0009105A9F584EC93E06CC4803BBFEB9B07CE
:1024C00021F483E0F801848339C088278115FBEA71
:1024D0009F0709F4ABCF81152FEB920791F381157C
:1024E0009F4779F38CE993E09F938F930E944F0568
:1024F00060EFD8018D919C910E94A6060F900F90DD
:102500008A3F910509F04CC462E0F8018081918115
:102510000E94A6068A3F910509F042C487CF80EC4D
:1025200093E09F938F930E944F050F900F90F801B7
:102530008281938181399B4A09F40CC4F80122817C
:1025400033812E3FFFEF3F0751F02D3F4FEF340710
:1025500049F02115310549F040E251E008C041E25F
:1025600051E005C04BE151E002C047E251E0D80123
:1025700014968C91813049F0823051F0833059F0BB
:10258000843061F08CE391E00BC080E391E008C0FF
:102590008DE291E005C083E391E002C081E491E027
:1025A0005F934F939F938F933F932F938CE893E088
:1025B0009F938F930E944F058AE0F80180877FC325
:1025C0000E947D2D9F938F9387E893E09F938F9335
:1025D0000E944F050F900F900F900F90D801149606
:1025E0008C91833031F0843079F0823009F07CC1F5
:1025F00006C068EFF801808191810E94A6060E94C2
:10260000DA1F0E94BA0C70C165EFD8018D919C91C0
:102610000E94A6066AEEF801808191810E94A606BA
:10262000BE016F5F7F4FC8010E94C80B80E893E036
:102630009F938F930E944F0568EED8018D919C91D6
:102640000E94A60660E0F801808191810E94A606A2
:1026500066EED8018D919C910E94A60666EEF80167
:10266000808191810E94A60666EED8018D919C9191
:102670000E94A606BE016F5F7F4FC8010E94C80B73
:102680000F900F908981882309F47AC08A8188236A
:1026900009F476C089E793E09F938F930E944F05DA
:1026A00066EEF801808191810E94A60668EED8014D
:1026B0008D919C910E94A60660E0F8018081918135
:1026C0000E94A60668EED8018D919C910E94A606F4
:1026D00063E0F801808191810E94A60668EED8012E
:1026E0008D919C910E94A60662E0F8018081918103
:1026F0000E94A60668EED8018D919C910E94A606C4
:1027000061E0F801808191810E94A60666EED80101
:102710008D919C910E94A60668EEF80180819181BE
:102720000E94A60663E0D8018D919C910E94A606A6
:1027300068EEF801808191810E94A60661E0D801CF
:102740008D919C910E94A60668EEF801808191818E
:102750000E94A60662E0D8018D919C910E94A60677
:1027600068EEF801808191810E94A60663E0D8019D
:102770008D919C910E94A60689E0F801848781C012
:1027800082E793E09F938F930E944F0563EFD801F8
:102790008D919C910E94A60668ECF8018081918140
:1027A0000E94A60663EFD8018D919C910E94A60617
:1027B00064E6F801808191810E94A60663EFD8014A
:1027C0008D919C910E94A60660E5F801808191811F
:1027D0000E94A606C8010E94EC0C292F30E00F9041
:1027E0000F902330310511F080E001C083E0D80163
:1027F0001C968C938BE693E09F938F930E944F05DA
:1028000063EFF801808191810E94A60668ECD801EF
:102810008D919C910E94A60663EFF80180819181C1
:102820000E94A60668ECD8018D919C910E94A60694
:1028300063EFF801808191810E94A60660E5D801CE
:102840008D919C910E94A606C8010E94EC0C292F34
:1028500030E00F900F902430310511F080E001C07E
:1028600084E0F801848781110EC084E693E09F9391
:102870008F930E944F0566EFD8018D919C910E9425
:10288000A6060F900F9064EFF801808191810E945D
:10289000A606BE016F5F7F4FC8010E94C80BD8011A
:1028A0001C968C91893049F0833051F0843059F076
:1028B000882361F083E291E00BC08FE491E008C0CF
:1028C00087E491E005C088E591E002C081E691E0EF
:1028D0009F938F9388E593E09F938F930E944F057A
:1028E0000F900F900F900F908BE0F80180870E945F
:1028F0007D2D9F938F9383E593E09F938F930E9409
:102900004F050F900F900F900F90D8018D919C91D3
:102910000E944A064C01019609F466C2F8018481BE
:10292000843069F18114910421F0FFEF8F16910436
:1029300069F40E94020C0E94EC228BE493E09F93C6
:102940008F930E944F050F900F904EC2823069F016
:10295000833081F0813009F047C2682DC8010E94A0
:10296000750D8F3F09F040C212C0682DC8010E944A
:102970004F0EF7CF682DC8010E94A70FF2CFF801C4
:10298000808191810E948B066C01019629F48CE074
:10299000D80118968C9328C2F801808191810E94F9
:1029A0008B067C01019699F3D8011C968C91FE014F
:1029B00031965F01853028F4833030F4882321F08C
:1029C000DEC08930A1F0DBC0D8011D969C911D9717
:1029D000987F282D2770922B1D969C9384FE02C011
:1029E000DD24DA9485FEC6C0FF24FA94C3C0F80142
:1029F0003585C401887499278834910509F0ABC0E6
:102A0000C1FEA9C0F0E38F229924959487949594F0
:102A1000879420E3C222DD2454E0D594C7945A95CC
:102A2000E1F7C828D92842E0C416D104E1F183E0D7
:102A3000C816D10409F478C0CA94CD2809F0C5C1DC
:102A4000E6FC17C0A701487055278E2D8F70E7FE52
:102A500007C0452B11F420E001C020EF822B0AC0F3
:102A6000452B11F420E001C020EF982F922B80E03D
:102A700002C080E090E0E4FE05C03860D8011D96F9
:102A80003C9303C0377FF8013587D8011D962C9100
:102A90001D97E5FE04C020611D962C9398C12F7EE2
:102AA000F801258794C1E0FE05C03064D8011D9669
:102AB0003C9303C03F7BF8013587D8011D968C916C
:102AC0001D97E1FE04C080681D968C9303C08F772C
:102AD000F8018587D8011D968C911D97E2FE04C0F0
:102AE00080621D968C9303C08F7DF8018587D80185
:102AF0001D968C911D97E3FE04C080641D968C93F7
:102B000003C08F7BF8018587D8011D968C911D9796
:102B1000E4FE04C080681D968C9303C08F77F80193
:102B2000858780E090E053C1C70124E095958795A3
:102B30002A95E1F7E7FE03C0806F90E003C0982F6D
:102B40009F7080E0387F2E2D2770E32EE22AD80177
:102B50001D96EC923CC1387F882D8770382BF80188
:102B6000358784FE02C0DD24DA9485FE4DC0FF2443
:102B7000FA944AC0833049F08430C9F045C08330AC
:102B800079F4E12CF12CC12CD12CD8018D919C91A0
:102B90000E948B068F3FBFEF9B07B1F1982F35C086
:102BA000843009F012C1E12CF12CC12CD12CF80198
:102BB000808191810E948B06AC018F3FFFEF9F07C0
:102BC00019F183FD02C080E001C080EF942F9F7057
:102BD000982BD8011D962C911D9744FF04C02860A6
:102BE0001D962C9303C0277FF8012587D8011D96D9
:102BF0002C911D9745FF04C020611D962C9305C0A4
:102C00002F7EF801258701C090E085E0D5011D9257
:102C10008A95E9F7F8018585898380E0F0E8CF1689
:102C2000D1044CF4960141E8C4164FEFD40624F4C5
:102C300021E83FEF01C02FE72A83A0E8EA16F1045C
:102C400054F49701B1E8EB16BFEFFB0614F421E84A
:102C50003FEF219501C021E82B83903811F0919529
:102C600001C09FE79C83803809F481E88D83C5010A
:102C70000E942F2089811F928F938D81282F082EEB
:102C8000000C330B3F938F938C81282F082E000C60
:102C9000330B3F938F938B81282F082E000C330B1F
:102CA0003F938F938A81282F082E000C330B3F937C
:102CB0008F938CE293E09F938F930E944F050FB602
:102CC000F894DEBF0FBECDBF8FC00E947D2D9F93B5
:102CD0008F9387E293E09F938F930E944F056EEF4F
:102CE000D8018D919C910E94A6060F900F900F9095
:102CF0000F908A3A910521F489E0F801808774C029
:102D00000E947D2D9F938F9382E293E09F938F93F8
:102D10000E944F05C8010E940B0C0E94020C0E94E9
:102D2000EC22D80118961C9200CB828185FF63CAE1
:102D3000D80118968C918B3009F05DCA88EF93E02A
:102D40009F938F930E944F058CE0F80180870F902E
:102D50000F9051CA60EFF801808191810E94A60610
:102D60008A3F9105A1F463E0D8018D919C910E9466
:102D7000A6068A3F910559F48CEB93E09F938F93BD
:102D80000E944F0583E0D80114968C9306C088EB0F
:102D900093E09F938F930E944F050F900F90CECB9F
:102DA00060EFF801808191810E94A6068A3F91051B
:102DB00009F03CCB63E0D8018D919C910E94A6065E
:102DC0008A3F910509F032CB7CCB90E080E025E092
:102DD000D5011D922A95E9F7F80125852983E12C73
:102DE000F12CC12CD12C1ECF81E00F900F900F90B1
:102DF0000F900F90DF91CF911F910F91FF90EF9067
:102E0000DF90CF90BF90AF909F908F90089588EC07
:102E100091E00E9483108AEB91E00C948310E8EC1F
:102E2000F1E08DE991E09183808313821282148214
:102E300015821086118612861386148615860E94C6
:102E4000020CEAEBF1E080E891E091838083138249
:102E500012821482158210861186128613861486B9
:102E600015860C94020C80910A030895CF93DF938A
:102E700000D01F92CDB7DEB720911804243021F581
:102E800023E029839B838A8382E08093E9008FEF8C
:102E90009091E800815095FD06C095ED9A95F1F767
:102EA00000008111F5CF8091E80085FF0DC040E062
:102EB00050E063E070E0CE0101960E94021C809118
:102EC000E8008E778093E8000F900F900F90DF91CD
:102ED000CF910895CF93DF9300D01F92CDB7DEB787
:102EE00020911804243061F519821A821B8222E095
:102EF00029838138910520F0805891099B838A832A
:102F000082E08093E9008FEF9091E800815095FD79
:102F100006C095ED9A95F1F700008111F5CF8091EB
:102F2000E80085FF0DC040E050E063E070E0CE01B6
:102F300001960E94021C8091E8008E778093E80041
:102F40000F900F900F90DF91CF910895209118046A
:102F5000243051F522E02093E9002FEF3091E80072
:102F6000215035FD06C035ED3A95F1F700002111ED
:102F7000F5CF2091E80025FF17C0209110012223F2
:102F800041F021E02093F10040E050E065E070E086
:102F900004C040E050E063E070E00E94021C8091B9
:102FA000E8008E778093E8000895CF93DF93209117
:102FB0001804243009F04AC0EC01809111018823E3
:102FC000E1F0809112018823C1F081E08093E90053
:102FD00081E8815049F09091E80095FD05C09AE2A2
:102FE0009A95F1F700C0F5CF8091E80085FF2EC0DB
:102FF00040E050E060E270E019C081E08093E900B9
:1030000081E8815059F09091E80095FD07C0EFE309
:10301000F1E03197F1F700C00000F3CF8091E800B4
:1030200085FF14C040E050E068E070E0CE010E94EF
:10303000021C8091E8008E778093E80080E2FE0118
:10304000AAEEB2E001900D928A95E1F7DF91CF915F
:103050000895CF93C091E801C1110BC00E94892D42
:10306000643C79408105910520F081E08093E8017E
:10307000C1E08C2FCF910895FF920F931F93CF93B0
:10308000DF93D82F0FB607FE83C0809118048430D9
:1030900081F08091030190E001962091050130E0DC
:1030A000822393232091040130E08217930709F0D3
:1030B000CBC00E942918811110C08091030190E0BB
:1030C00001962091050130E0822393232091040191
:1030D00030E08217930709F0B7C00E947D2D8C0164
:1030E000C091E900CF709091EC00892F817090FD24
:1030F00080E8C82B83E08093E90085E0F82E80917A
:10310000EB0085FD42C08091EB0080FF3EC08091C6
:10311000EE0087FF3AC08091040190910301981757
:1031200009F457C09091E80095FF8CC0E09101012F
:10313000F0910201E80FF11D20818F5F9091050150
:103140008923809304012093F1008091E80085FD9C
:10315000E2CF8091E80080FFDECF8091E8008E779B
:103160008093E800F0920001D6CF8091030190E0B7
:1031700001962091050130E08223932320910401E0
:1031800030E08217930709F44AC0CF70C093E9007A
:1031900040910301842F90E001962091050130E0D9
:1031A000822393232091040130E08217930709F4CE
:1031B0004EC0E0910101F0910201E40FF11DD083B6
:1031C000809103018F5F9091050189238093030112
:1031D0003EC08091E80085FF35C0D093F10081E0CA
:1031E0002091F2003091F300232B91F09091E800B0
:1031F00090FF0EC09091E80095FF03C01092F1007F
:10320000F9CF9091E8009E779093E800F09200014A
:10321000882309F4AACFCF70C093E90018C0809129
:103220000001882309F4B1CF0E947D2D9C018017F5
:10323000910711F4890163CF90910001915090930F
:103240000001F8CF80E0CCCF40910301B2CF80E005
:10325000DF91CF911F910F91FF90089580911704F6
:10326000811104C00E946A1E0C94CC1E0895109215
:1032700017040895089542E261EC81E00E947B1BEF
:1032800042E061EC82E00E947B1B42E261EC83E061
:103290000C947B1B80911A04833009F453C030F4E2
:1032A000813071F0823009F4BAC008958A3009F48F
:1032B000A6C08B3009F478C0893009F0C8C020C09E
:1032C00080911904813A09F0C2C08091E800877F9B
:1032D0008093E80080911D0490911E04892B21F4B5
:1032E00060E28AEE92E003C060E080E090E070E08F
:1032F0000E944F1C8091E8008B778093E80008952E
:1033000080911904813209F0A2C080911D0490912E
:103310001E04892B09F09BC08091E800877F809371
:10332000E8008091E80082FD05C0809118048111B9
:10333000F8CF8DC08091F10080930A038091E8005E
:103340008B7781C080911904813A09F080C0809107
:103350001D0490911E04892BA1F48091E800877FC1
:103360008093E8008091E80080FFFCCF80911101FC
:103370008093F1008091E8008E778093E8000E94AE
:10338000B01B80911D0490911E04019709F05FC04D
:103390008091E800877F8093E8008091E80080FFBB
:1033A000FCCF809110014AC080911904813209F04C
:1033B0004EC080911D0490911E04892B69F4809168
:1033C000E800877F8093E8000E94B01B80911B0477
:1033D000809311010E94EC2280911D0490911E04A3
:1033E0000197A9F58091E800877F8093E8000E940B
:1033F000B01B80911B04809310010C94EC228091EF
:103400001904813221F58091E800877F8093E800DC
:103410000E94B01B80911C0480930B03089580913F
:103420001904813AA1F48091E800877F8093E80035
:103430008091E80080FFFCCF80910B038093F10026
:103440008091E8008E778093E8000C94B01B08957B
:1034500080910A038093E90110920A030E948E0C66
:103460000C94EC220C94281A0E94292D80911604A9
:10347000882329F00E94362D81110C94651B089534
:103480000E944B2D8091E90180930A0308950C94CA
:10349000401A08950C94491ACF9384B7877F84BF4C
:1034A0000FB6F894A89580916000886180936000C1
:1034B000109260000FBE90E080E80FB6F894809301
:1034C0006100909361000FBE8CE398E10E94E82CAC
:1034D00086E091E00E94D51F80EE95E00E94B60440
:1034E0000E94760C0E9494200E946A1E0E94CC1EAC
:1034F00078940E94962080911804843029F00E94CC
:10350000BA1F0E94491AF7CF8EEC95E00E94B604CC
:103510000E944A1A80EC95E00E94B604C3E08091B4
:103520001804853019F40E94341AF9CF0E94122D24
:103530000E949A202091E4003091E5008091E601FC
:103540009091E7012817390709F466C08091E400DB
:103550009091E5009093E7018093E6010E9429187D
:10356000882309F459C080911804843009F054C0AC
:103570008091E9008F702091EC00922F917020FDD6
:1035800090E8892BC093E9009091EB0090FF41C037
:103590009091EE0097FF3DC09091040120910301AE
:1035A000291709F12091E80025FF1DC0E0910101D4
:1035B000F0910201E90FF11D30819F5F209105011B
:1035C0009223909304013093F1009091E80095FDCF
:1035D000E3CF9091E80090FFDFCF9091E8009E77D5
:1035E0009093E800D9CF2091F2003091F300232B83
:1035F00081F09091E80090FF0CC09091E80095FF59
:1036000003C01092F100F9CF9091E8009E7790935B
:10361000E8008F708093E9000E94BA1F80CF292FA5
:10362000332723303105C9F060F42130310581F0B2
:103630002230310509F041C084E590E02DE336E009
:1036400040C021323105E1F02232310531F135C07F
:1036500082E190E021E936E034C09927813091057C
:1036600049F028F0029749F5E9EFF5E005C0E9E3F4
:10367000F6E002C0EFE2F6E0849190E09F0121C005
:1036800063307105D0F4660F771FFB01EE58FE4FD3
:103690002081318189E090E014C06330710568F4C5
:1036A000FB01EE0FFF1FE459FE4F20813181FB012A
:1036B000E759FE4F808190E004C080E090E020E078
:1036C00030E0FA0131832083089584E189BD86E1E9
:1036D00089BD09B400FEFDCF8091D8008F7D809315
:1036E000D8008091E00082608093E0008091E0004B
:1036F00081FDFCCF0895982F973068F59093E900ED
:10370000981739F07091EC002091ED005091F00085
:1037100003C0242F762F50E021FD02C09F5FECCF25
:103720003091EB003E7F3093EB003091ED003D7F18
:103730003093ED003091EB0031603093EB007093EB
:10374000EC002093ED005093F0002091EE0027FD57
:10375000E5CF80E008958F708093E90081E00895BF
:103760008091190487FF11C08091E80082FD05C097
:10377000809118048111F8CF11C08091E8008B77F7
:103780000BC080911804882349F08091E80080FFE5
:10379000F8CF8091E8008E778093E800089520911B
:1037A000E4003091E50095E64091EC00842F8170B3
:1037B00040FF23C08091E80080FD1DC08091180467
:1037C000882399F0853099F08091EB0085FD11C038
:1037D0004091E4005091E5002417350729F39150FA
:1037E00011F09A01E1CF84E0089582E0089583E02A
:1037F000089581E0089580E008954091E80042FF37
:10380000DDCF0895CF92DF92EF92FF920F931F9337
:10381000CF93DF93EC018B017A010E94CF1B8111C2
:1038200035C0E114F10439F0F70180819181081B62
:10383000190BC80FD91FC12CD12C0115110529F165
:103840008091E80085FD18C08091E8008E77809314
:10385000E8000E94BA1FE114F10449F0F7018081E9
:103860009181C80ED91ED182C08285E00FC00E940E
:10387000CF1B882311F30AC089918093F100015076
:103880001109FFEFCF1ADF0AD8CF80E0DF91CF9187
:103890001F910F91FF90EF90DF90CF9008952091AE
:1038A0001F04309120042617370748F06115710571
:1038B00039F42091E8002E772093E80001C0B90187
:1038C000FC0120E06115710569F1809118048823DD
:1038D000E1F18530E1F18091E80083FD3AC080910B
:1038E000E80082FD2CC08091E80080FFEBCF809142
:1038F000F2009091F3006115710551F08830910547
:1039000038F421912093F100615071090196F3CFB1
:1039100021E0089709F020E08091E8008E778093FD
:10392000E800D0CF2111D1CF0AC08091180488239C
:1039300061F0853061F08091E80083FD0AC08091DC
:10394000E80082FFF2CF80E0089582E0089583E0EE
:10395000089581E0089520911F04309120042617D6
:10396000370748F06115710539F42091E8002E778A
:103970002093E80001C0B901FC0120E06115710548
:1039800081F180911804882309F43EC0853009F440
:103990003DC08091E80083FD3BC08091E80082FD3E
:1039A0002DC08091E80080FFE9CF8091F2009091D6
:1039B000F3006115710559F08830910540F42491A8
:1039C0002093F1003196615071090196F2CF21E008
:1039D000089709F020E08091E8008E778093E80056
:1039E000CDCF2111CECF0AC080911804882361F079
:1039F000853061F08091E80083FD0AC08091E80085
:103A000082FFF2CF80E0089582E0089583E0089578
:103A100081E008951F93CF93DF93CDB7DEB7AA97C8
:103A20000FB6F894DEBF0FBECDBFE9E1F4E08091A0
:103A3000F100819324E0E132F207C9F70E944A19AC
:103A40008091E80083FF2EC18091190490911A049F
:103A5000492F50E04A30510508F024C1FA01E95CD1
:103A6000FE4F0C94DF31803821F0823809F01AC102
:103A700008C08091150490911604992389F0826002
:103A80000FC080911D048F70873008F00BC18093A8
:103A9000E9008091EB0085FB882780F91092E9000E
:103AA0009091E800977F9093E8008093F100109246
:103AB000F100D1C0282F2D7F09F0F4C0882319F020
:103AC000823061F0EFC080911B04813009F0EAC0C0
:103AD000933009F080E0809316042EC080911B047F
:103AE00081112AC080911D048F702FEF280F26307E
:103AF00008F0D8C08093E9002091EB0020FF1CC0A3
:103B0000933021F48091EB00806214C09091EB001F
:103B100090619093EB0021E030E0A90102C0440FD6
:103B2000551F8A95E2F74093EA001092EA008091CF
:103B3000EB0088608093EB001092E9008091E80030
:103B4000877F8093E8000E94B01BACC08111AAC09F
:103B500010911B041F778091E3008078812B809364
:103B6000E3008091E800877F8093E8000E94B01B0B
:103B70008091E80080FFFCCF8091E3008068809313
:103B8000E300111102C082E001C083E080931804B9
:103B900089C08058823008F085C080911B049091C4
:103BA0001C048C3D53E0950779F583E08A838AE213
:103BB00089834FB7F894DE01139620E03EE051E28E
:103BC000E32FF0E050935700E49120FF03C0E2950B
:103BD000EF703F5FEF708E2F90E0EA3010F0C796E5
:103BE00001C0C0968D939D932F5F243149F74FBF3D
:103BF0008091E800877F8093E8006AE270E0CE0160
:103C000001960E944F1C16C060911D0470911E0405
:103C1000AE014F5F5F4F0E940F1BBC01892B09F45F
:103C200041C09091E800977F9093E80089819A8144
:103C30000E94AB1C8091E8008B778093E80032C033
:103C4000803881F58091E800877F8093E80080913B
:103C500014048093F1008091E8008E7772CF811177
:103C600021C080911B0490911C0499270297D4F4E1
:103C70008091E800877F8093E80080911B04809307
:103C800014040E94B01B80911404811106C080911D
:103C9000E30087FD02C081E001C084E08093180446
:103CA0000E943B198091E80083FF0AC08091E800E0
:103CB000877F8093E8008091EB0080628093EB0027
:103CC000AA960FB6F894DEBF0FBECDBFDF91CF919D
:103CD0001F9108950E94DB1E0E94E31EE0EEF0E0BB
:103CE000808181608083E8EDF0E080818F77808340
:103CF00019BCA7EDB0E08C918E7F8C9380818F7E74
:103D000080831092170408950F931F93CF93DF932E
:103D10000E94DB1E0E94E31EC8EDD0E088818F77F1
:103D2000888388818068888388818F7D8883E7ED98
:103D3000F0E080818068808319BC10921804109292
:103D40001404109216041092150400EE10E0F8010D
:103D500080818B7F808388818160888342E060E0FE
:103D600080E00E947B1BE1EEF0E080818E7F80830B
:103D7000E2EEF0E0808181608083808188608083D2
:103D8000F80180818E7F8083888180618883DF91C4
:103D9000CF911F910F910895E8EDF0E080818F7E23
:103DA0008083E7EDF0E080818160808381E0809313
:103DB00017040C94841EE8EDF0E080818C7F8083F2
:103DC0001092E20008951092DA001092E100089536
:103DD0001F920F920FB60F9211240BB60F922F93D2
:103DE0003F934F935F936F937F938F939F93AF9383
:103DF000BF93EF93FF938091E10082FF0BC080910E
:103E0000E20082FF07C08091E1008B7F8093E10098
:103E10000E94B91F8091DA0080FF1FC08091D800F6
:103E200080FF1BC08091DA008E7F8093DA00809142
:103E3000D90080FF0DC084E189BD86E189BD09B448
:103E400000FEFDCF81E0809318040E942E1905C06A
:103E500019BC109218040E9437198091E10080FF6C
:103E600019C08091E20080FF15C08091E2008E7F32
:103E70008093E2008091E20080618093E200809173
:103E8000D80080628093D80019BC85E08093180424
:103E90000E94321A8091E10084FF30C08091E200DC
:103EA00084FF2CC084E189BD86E189BD09B400FE90
:103EB000FDCF8091D8008F7D8093D8008091E10064
:103EC0008F7E8093E1008091E2008F7E8093E200FC
:103ED0008091E20081608093E20080911404882345
:103EE00011F084E007C08091E30087FD02C081E00B
:103EF00001C083E0809318040E94471A8091E1007A
:103F000083FF24C08091E20083FF20C08091E10004
:103F1000877F8093E10082E080931804109214045C
:103F20008091E1008E7F8093E1008091E2008E7F9E
:103F30008093E2008091E20080618093E20042E0A1
:103F400060E080E00E947B1B0E943A19FF91EF9194
:103F5000BF91AF919F918F917F916F915F914F91A1
:103F60003F912F910F900BBE0F900FBE0F901F909F
:103F700018950895CF93809118048823A1F0C091DB
:103F8000E900CF709091EC00892F817090FD80E85E
:103F9000C82B1092E9008091E80083FD0E940A1D61
:103FA000CF70C093E900CF9108959093110380934F
:103FB00010030895E0911003F0911103309721F060
:103FC0000190F081E02D099480E00895EF92FF9236
:103FD0000F931F93CF93DF93E0911003F0911103A0
:103FE0003097B1F18C010280F381E02D0995809129
:103FF000060482FF2DC080FF04C083EA97E00E9480
:10400000B604E80110E28DE9E82E87E0F82E8091F1
:10401000060480FF0BC088811F928F93FF92EF925E
:104020000E944F050F900F900F900F901150219606
:104030001111EDCF8091060480FF0AC08BE997E053
:10404000DF91CF911F910F91FF90EF900C94B604E8
:10405000DF91CF911F910F91FF90EF900895E09124
:104060001003F0911103309721F00480F581E02DC9
:1040700009940895CF93DF9320910E0330910F039D
:104080002817390709F190930F0380930E03E091ED
:104090001003F09111033097B9F0EC010680F7811D
:1040A000E02D09958091060482FF0EC080FF0CC0B0
:1040B000DF93CF938DE897E09F938F930E944F05F6
:1040C0000F900F900F900F90DF91CF910895CF93A5
:1040D000DF9320910C0330910D032817390709F164
:1040E00090930D0380930C03E0911003F091110362
:1040F0003097B9F0EC010084F185E02D09958091AD
:10410000060482FF0EC080FF0CC0DF93CF938DE7C3
:1041100097E09F938F930E944F050F900F900F9001
:104120000F90DF91CF9108950C9455210E94742D2A
:104130000C947E0C8F929F92AF92BF92CF92DF929F
:10414000EF92FF920F931F93CF93DF9300D000D095
:104150001F92CDB7DEB70E94071703E113E0F12CE1
:104160008F2D0E94850C4C01F801A080B180A826FB
:10417000B926A114B10439F4F3940E5F1F4FF8E08F
:10418000FF12EECF39C08091060481FD0E946921A3
:10419000E12CCC24C394D12CC5018C219D21892BE9
:1041A00021F1E982FA8221E0C4018C219D21892B31
:1041B00009F420E02B830E947D2D8160782F9D8360
:1041C0008C8349815A816B818D810E949F21498115
:1041D0005A816B817C818D810E94142DF801808130
:1041E00091818C259D2591838083E394CC0CDD1CEB
:1041F000F0E1EF12D1CFC0CF8FEF89838A831B828A
:104200000E947D2D8160782F9D838C8349815A8106
:104210006B818D810E949F210E94132D0E94E92FA6
:104220000E94DA1F90911203891759F10E94DA1F38
:10423000809312039091060492FF0EC090FF0CC071
:104240001F928F938EEA97E09F938F930E944F0562
:104250000F900F900F900F90809112030F900F907E
:104260000F900F900F90DF91CF911F910F91FF90C2
:10427000EF90DF90CF90BF90AF909F908F900C9475
:10428000252D0F900F900F900F900F90DF91CF91F1
:104290001F910F91FF90EF90DF90CF90BF90AF9064
:1042A0009F908F9008950C94BA0C0895CF93C62FC9
:1042B0000E94850C21E030E002C0220F331FCA9516
:1042C000E2F72823392381E0232B09F480E0CF9102
:1042D0000895EF92FF920F931F93CF93DF9385EC96
:1042E00097E00E94B604C0E0D0E080E2E82E81E0D2
:1042F000F82E09EB17E08C2F0E94850C0E94FF2CF2
:10430000FF92EF929F938F93DF93CF931F930F931F
:104310000E944F0521968DB79EB708960FB6F89468
:104320009EBF0FBE8DBFC830D10529F7DF91CF9159
:104330001F910F91FF90EF90089508950895CF93E6
:10434000DF93CDB7DEB72B970FB6F894DEBF0FBE65
:10435000CDBF942F4F83252F588769877A878B8706
:104360004A855B85452B31F02F3F31F481E09F3F3B
:1043700019F403C081E001C080E080FD07C04F81D7
:10438000588569857A858B850E94142DDE011196EA
:1043900086E0FD0111928A95E9F785E0FE013796E6
:1043A00001900D928A95E1F749815A816B817C8158
:1043B0008D819E810E9405292B960FB6F894DEBF51
:1043C0000FBECDBFDF91CF910895882309F4BBC004
:1043D0009CEF980F913A18F40E94E32B0DC090E2E5
:1043E000980F983058F4877091E001C0990F8A9522
:1043F000EAF7892F0E94882C0C94C22C9BE5980F19
:10440000933070F4853A29F0863A31F083E890E0F1
:1044100005C081E890E002C082E890E00C943A2068
:1044200098E5980F973108F08EC0883A09F445C096
:10443000893A09F445C08A3A09F445C08B3A09F42F
:1044400045C08C3A09F445C08D3A09F445C08E3A0E
:1044500009F445C08F3A09F445C0813B09F445C0D1
:10446000803B09F445C0823B09F445C0833B09F415
:1044700045C0843B09F445C0853B09F445C0863BF3
:1044800009F445C0873B09F445C0883B09F445C0A1
:10449000893B09F445C08A3B09F445C08B3B09F4CC
:1044A00045C08C3B09F445C08D3B09F445C08E3BAB
:1044B00009F445C080E090E044C082EE90E041C045
:1044C00089EE90E03EC08AEE90E03BC085EB90E044
:1044D00038C086EB90E035C083EB90E032C084EBCF
:1044E00090E02FC087EB90E02CC08CEC90E029C0CE
:1044F0008DEC90E026C083E891E023C08AE891E04B
:1045000020C082E991E01DC084E991E01AC081E2F7
:1045100092E017C083E292E014C084E292E011C0FE
:1045200085E292E00EC086E292E00BC087E292E064
:1045300008C08AE292E005C08FE690E002C080E702
:1045400090E00C9467200895882329F19CEF980F40
:10455000913A18F40E94332C0DC090E2980F9830D5
:1045600058F4877091E001C0990F8A95EAF7892F76
:104570000E948E2C0C94C22C9BE5980F933020F453
:1045800080E090E00C943A20885A873120F480E053
:1045900090E00C9467200895882321F00E94882CD5
:1045A0000C94C22C0895882321F00E948E2C0C9428
:1045B000C22C08950E94A82C0E94772C0E94C22C25
:1045C0000E948E300E945C2F80E090E00E943A2092
:1045D00080E090E00C9467200E94982C0C94DA22E2
:1045E000CF92DF92EF92FF920F931F93CF93DF93BF
:1045F00000D000D01F92CDB7DEB76C010E94272DEE
:10460000811118C385E0F601DE01119601900D922B
:104610008A95E1F7F601408151812381348121158A
:10462000310531F05F3F31F481E04F3F19F403C0B1
:1046300081E001C080E080FDFDC2F601F280E580EE
:10464000E2948FE0E82249835A83FB82722F3D83F4
:104650002C836F2D8D810E945F2B8C010E945E2B1D
:104660000E94582AE12FE295EF708E2F90E0FC0116
:10467000EF5BFE4F0C94DF31812F807F1F7088230A
:1046800011F01295107FFF20B9F0112329F0812F2E
:104690000E949B2C0E94C22C802F0F900F900F9095
:1046A0000F900F90DF91CF911F910F91FF90EF909E
:1046B000DF90CF900C94E521802F0E94A42211233B
:1046C00009F4B8C2812F0E94A12C0F900F900F9077
:1046D0000F900F90DF91CF911F910F91FF90EF906E
:1046E000DF90CF900C94C22C812F807F1F7080327E
:1046F00011F01295107F002319F0013009F12BC041
:10470000FF20A9F0EE2059F1F1E0812FEF1228C02F
:104710000F900F900F900F900F90DF91CF911F91FE
:104720000F91FF90EF90DF90CF900C94AB2CEE2088
:1047300021F021E0E21609F47DC20E94AE2C4DC0AA
:10474000FF20E9F085E08E1508F474C20E94852CE4
:10475000812329F042C0FF20F1F1E11015C0812F23
:104760000F900F900F900F900F90DF91CF911F91AE
:104770000F91FF90EF90DF90CF900C94CC2294E0BB
:104780009E1508F457C229C0F601858180FF13C029
:104790008F708583E4CF003F09F489C108F055C1CB
:1047A00080E4800F803208F459C1FF2009F4EAC187
:1047B000EE2009F49AC1802F0E94E521093309F007
:1047C000DAC1FFEF21EE84E0F15020408040E1F7B4
:1047D00000C000002FC2E110D7C1812F59C1812F25
:1047E00086958695837019F08130B9F023C2FF2039
:1047F00019F0C801937002C080E090E00F900F9014
:104800000F900F900F90DF91CF911F910F91FF901C
:10481000EF90DF90CF900C943A20FF2019F0C80160
:10482000937002C080E090E00F900F900F900F9077
:104830000F90DF91CF911F910F91FF90EF90DF903C
:10484000CF900C946720802FFF2019F00E946F2ECC
:1048500002C00E94D72E0F900F900F900F900F90D4
:10486000DF91CF911F910F91FF90EF90DF90CF904C
:104870000C945C2F812F837009F070C0F110DAC1A5
:10488000202F229526952770220F220F602F6F7000
:10489000862F90E0A0E0B0E06C017D01022E04C004
:1048A000CC0CDD1CEE1CFF1C0A94D2F704FF12C0D6
:1048B0008FE090E0A0E0B0E004C0880F991FAA1F2D
:1048C000BB1F2A95D2F7BC01CD01609570958095EC
:1048D000909503C060E070E0CB01169516951370BB
:1048E0001230B1F040F56C297D298E299F291130B5
:1048F00031F10F900F900F900F900F90DF91CF91AB
:104900001F910F91FF90EF90DF90CF900C94732A3E
:104910006C297D298E299F290F900F900F900F9061
:104920000F90DF91CF911F910F91FF90EF90DF904B
:10493000CF900C948D2A0E94732AC701B6010F9064
:104940000F900F900F900F90DF91CF911F910F91CB
:10495000FF90EF90DF90CF900C94592AFF2019F030
:10496000812F817001C08695882309F463C1202FAF
:10497000229526952770220F220F602F6F70862FA9
:1049800090E0A0E0B0E06C017D01022E04C0CC0CF0
:10499000DD1CEE1CFF1C0A94D2F704FF12C08FE04E
:1049A00090E0A0E0B0E004C0880F991FAA1FBB1FD1
:1049B0002A95D2F7BC01CD016095709580959095B0
:1049C00003C060E070E0CB011695169513701230AD
:1049D000B1F040F56C297D298E299F29113031F1E4
:1049E0000F900F900F900F900F90DF91CF911F912C
:1049F0000F91FF90EF90DF90CF900C943A2B6C29A1
:104A00007D298E299F290F900F900F900F900F9066
:104A1000DF91CF911F910F91FF90EF90DF90CF909A
:104A20000C944C2B0E943A2BC701B6010F900F90AB
:104A30000F900F900F90DF91CF911F910F91FF90EA
:104A4000EF90DF90CF900C94282B023F09F45EC0CA
:104A500008F449C0033F09F46CC0A7CE902F9071B1
:104A6000E92E812F8F71FF2051F00E94C12A802FE3
:104A7000EE2019F08295807F73CE8F7071CE0E94E8
:104A8000E22A802FEE2019F08295807F01C08F707E
:104A90000F900F900F900F900F90DF91CF911F917B
:104AA0000F91FF90EF90DF90CF900C94D322FF20D6
:104AB000A9F0E4E0EE1508F4BDC0812F8F710F90CE
:104AC0000F900F900F900F90DF91CF911F910F914A
:104AD000FF90EF90DF90CF900C94072BF5E0FE1540
:104AE00008F4A8C0EACFFF2099F0812F8F710F90B2
:104AF0000F900F900F900F90DF91CF911F910F911A
:104B0000FF90EF90DF90CF900C94C12AFF2069F3C3
:104B1000812F8F710F900F900F900F900F90DF915A
:104B2000CF911F910F91FF90EF90DF90CF900C9459
:104B3000E22AFF2089F0812F8F710F900F900F9044
:104B40000F900F90DF91CF911F910F91FF90EF90F9
:104B5000DF90CF900C94AC2A0F900F900F900F9095
:104B60000F90DF91CF911F910F91FF90EF90DF9009
:104B7000CF900C94A72A033509F423CE073409F00B
:104B800059C01FCEEE2021F2802F0F900F900F9072
:104B90000F900F90DF91CF911F910F91FF90EF90A9
:104BA000DF90CF900C94A422412F4F70602FC6014C
:104BB0000E94E92D0F900F900F900F900F90DF91B2
:104BC000CF911F910F91FF90EF90DF90CF900C94B9
:104BD000B32901112FC0FF2069F10E94EC222FEFB1
:104BE00080E792E0215080409040E1F700C0000053
:104BF0000F900F900F900F900F90DF91CF911F911A
:104C00000F91FF90EF90DF90CF900C94CA2D412F21
:104C10004F70602FC6010F900F900F900F900F9064
:104C2000DF91CF911F910F91FF90EF90DF90CF9088
:104C30000C94EC2D0F900F900F900F900F90DF9130
:104C4000CF911F910F91FF90EF90DF90CF9008953B
:104C50001F93CF93DF9300D000D01F92CDB7DEB764
:104C6000942F4983252F5A836B837C838D834C81BA
:104C70005D81452B31F02F3F31F481E09F3F19F4E6
:104C800003C081E001C080E0182F117080FD24C0B6
:104C900049815A816B817C818D810E945F2B292FF4
:104CA00022952F702C3030F42A3048F422502230D4
:104CB00068F013C02C3061F02F3051F00EC0803CF2
:104CC00028F0803E50F0815F833038F011E005C05D
:104CD00093FB112710F901C010E0812F0F900F9066
:104CE0000F900F900F90DF91CF911F910895CF9368
:104CF000DF9300D000D01F92CDB7DEB70F900F909A
:104D00000F900F900F90DF91CF910895CF93DF9385
:104D100000D000D000D0CDB7DEB726960FB6F894FD
:104D2000DEBF0FBECDBFDF91CF9108951F93CF930C
:104D3000DF93C091230316E080912403C81799F0F4
:104D4000D0E01C9FF0011D9FF00D1124EB5DFC4F86
:104D50004081518162817381848195810E94862680
:104D60002196C770E9CFDF91CF911F9108954091AF
:104D700055035091560360915703709158038091E9
:104D8000590390915A030C9486260F931F93CF9347
:104D9000DF9380915A0382958F7009F05DC08091F6
:104DA0005703882309F458C08091230310912403EA
:104DB0006091550370915603C0915803D0915903E7
:104DC00091E06F3F09F090E0292F06E0811709F488
:104DD00043C0209721F07F3F21F030E003C031E055
:104DE00001C0322F90E030FD34C0089FF001099FD0
:104DF000F00D1124DF01AB5DBC4F11963C91119772
:104E0000371327C03C91361324C012963C91129759
:104E100031111FC013964D915C9114974C1B5D0B83
:104E2000483C5105B0F480915A038F7080618093A3
:104E30005A03E65DFC4F80818F708061808385E539
:104E400093E00E94F022DF91CF911F910F910C947B
:104E5000962601968770BACFDF91CF911F910F915F
:104E600008959F92AF92BF92CF92DF92EF92FF92FE
:104E70000F931F93CF93DF93CDB7DEB761970FB634
:104E8000F894DEBF0FBECDBF8C0185E0F801DE01D6
:104E90001D9601900D928A95E1F7F80140815181AC
:104EA000F280C380D4809091550360915603209185
:104EB0005803309159032115310531F06F3F31F41A
:104EC00081E09F3F19F403C081E001C080E0F82F2A
:104ED000F1709F2E80FD52C185E5A82E83E0B82E8B
:104EE000E0905703F601E21BF30BEE2009F4E8C053
:104EF00080915A03E83CF10508F0A4C0282F207FD8
:104F000009F053C0561313C0491311C0EF2CF11010
:104F10000EC08F70806180935A030E94B726C5012E
:104F20000E94F02280915A03F80185835BC1C1146D
:104F3000D10431F05F3F31F481E04F3F19F403C0F9
:104F400081E001C080E080FD03C081E08F2502C0C8
:104F500080E090E0F82FF170EF2E80FF1CC0809170
:104F600023032091240336E0821709F418C190E04E
:104F7000389FF001399FF00D1124EB5DFC4F6181EA
:104F8000561306C06081461303C06281F61203C047
:104F900001968770E9CFEF2CFF2009F423C180919F
:104FA0005A03816080935A0362C0561306C04913A6
:104FB00004C0F11002C0F801A7C04D875E87FF86CC
:104FC0007C2DD98AC88A6F2D89890E94282688233A
:104FD00099F1FF2089F120915A03822F82958F70D9
:104FE00090E0029774F08091550390915603988752
:104FF0008F831986DB86CA862C87CE0107960E948E
:10500000F02286E0F801A5E5B3E001900D928A95C3
:10501000E1F70E94C5260E94B72611C0561749F134
:105020004D875E87FF867C2DD98AC88A6F2D898936
:105030000E94282681112CC0C8010E94F022EE2473
:10504000E394D0C0282F207F49F77C2DD98AC88AC5
:105050006F2D89890E94772685E593E00E94F022D2
:1050600086E0F50111928A95E9F70E94B726E12CB6
:10507000B9C04913D5CFF110D3CFF8018583C8014A
:105080000E94F02286E0F50111928A95E9F7AAC004
:10509000FF2091F220915A03822F82958F7090E029
:1050A00002970CF4AECF80915503909156039A83EA
:1050B00089831B82DD82CC822E83CE0101969FCF15
:1050C000E83CF10508F04BC0EF2CFF2009F4B4CF09
:1050D000561330C049132EC020915A0320FD21C021
:1050E000822F82958F70482F50E041155105C9F0ED
:1050F000F80125834F30510541F08F5F982F92952D
:10510000907F822F8F70892B8583C8010E94F022A7
:1051100086E0F801A5E5B3E001900D928A95E1F7EC
:105120002AC086E0F801A5E5B3E001900D928A95CA
:10513000E1F758C04D875E87FF867C2DD98AC88AE3
:105140006F2D89890E94282681115BCF80915A0397
:10515000816080935A03C8010E94F02243C07C2DD5
:10516000D98AC88A6F2D89890E94772686E0F50141
:1051700011928A95E9F70E94B72634C0FF2009F4FE
:105180005BCF4D875E87FF867C2DD98AC88A6F2DBD
:1051900089890E942826882309F44ECF32CF7C2D9E
:1051A000D98AC88A6F2D89890E945F2B292F229561
:1051B0002F70223028F49F7039F0811105C00BC088
:1051C000243028F49F7049F4805E883020F0C801B4
:1051D0000E94F0229E2CE92C05C0F8019581907F59
:1051E00099F7F9CF8E2D61960FB6F894DEBF0FBEFA
:1051F000CDBFDF91CF911F910F91FF90EF90DF9086
:10520000CF90BF90AF909F9008951F93CF93DF935F
:10521000CDB7DEB72C970FB6F894DEBF0FBECDBF6B
:105220004F83588769877A878B879C87CE0107963B
:105230000E9431278823D1F09F8188852A853B856C
:10524000232B31F08F3F31F481E09F3F19F403C0ED
:1052500081E001C080E080FD47C04F8158856985AD
:105260007A858B859C850E9486263EC086E0FE015D
:105270003796DE01119601900D928A95E1F7FF8134
:10528000E8856A857B856115710531F0EF3F31F462
:1052900081E0FF3F19F403C081E001C080E080FDA0
:1052A00023C02091240330E0C9010196877099271B
:1052B0004091230350E084179507F1F1F983EA83C5
:1052C0007D836C8396E0929FD001939FB00D112453
:1052D000AB5DBC4FFE01319601900D929A95E1F7BE
:1052E000809324030E94962616E0809123039091D8
:1052F0002403891771F1189FC00111248B5D9C4F05
:105300000E943127882329F1E09123031E9FF00199
:105310001124EB5DFC4F4081518162817381848156
:1053200095810E9486268091230390E001968770E4
:10533000992780932303D9CF0E94EC221092240353
:1053400010922303E5E5F3E086E0DF011D928A95E4
:10535000E9F72C960FB6F894DEBF0FBECDBFDF91F4
:10536000CF911F910895DF92EF92FF920F931F93B9
:10537000CF93DF93FC01892B09F488C0E12CF12C39
:10538000DD24D394EF0121968491853709F460C020
:1053900058F4843708F04EC0843008F068C081307B
:1053A000D1F0823071F172C0883709F45BC050F4DB
:1053B000863709F453C0873709F068C08E2D0E94E4
:1053C000952C52C09CE7980F903708F05FC08F77FC
:1053D0000E94A4224EC08F010E5F1F4FFE018491D8
:1053E00090E2980F983050F48770FD2D01C0FF0FA8
:1053F0008A95EAF78F2F0E949B2C15C00E94E52109
:1054000014C08F010E5F1F4FFE01849190E2980F30
:10541000983068F48770FD2D01C0FF0F8A95EAF778
:105420008F2F0E94A12C0E94C22CE80122C00E9452
:10543000A422FBCFCF010296FE01C491CC2361F0E0
:10544000EFE9FFE03197F1F700C00000C150F6CF5F
:10545000CF010296FE01F490EC010BC00E94852C56
:10546000E82E07C00E94982C0E94C22C02C00E9405
:10547000E5218F2D882341F0EFE9FFE03197F1F727
:1054800000C000008150F6CFFE017CCFDF91CF91AC
:105490001F910F91FF90EF90DF9008956093DB03D1
:1054A0007093DC038093DD039093DE030C94242D32
:1054B00008950F931F930091DF031091E003209153
:1054C000E1033091E203602B712B822B932B6093CD
:1054D000DF037093E0038093E1039093E2031F9155
:1054E0000F910C94232D0F931F930091DF031091C4
:1054F000E0032091E1033091E203602371238223D2
:1055000093236093DF037093E0038093E103909310
:10551000E2031F910F910C94232D0F931F93009181
:10552000DF031091E0032091E1033091E203602753
:105530007127822793276093DF037093E0038093A2
:10554000E1039093E2031F910F910C94232D60E0EF
:1055500070E0CB010C944E2A0F931F9341E050E072
:1055600060E070E08A019B0104C0000F111F221F40
:10557000331F8A95D2F7C901B8011F910F910C947E
:105580004E2A0F931F9341E050E060E070E004C0AA
:10559000440F551F661F771F8A95D2F78091DB0352
:1055A0009091DC03A091DD03B091DE038A019B01A1
:1055B000082B192B2A2B3B2BC901B8011F910F91E6
:1055C0000C944E2A0F931F9341E050E060E070E08E
:1055D00004C0440F551F661F771F8A95D2F7409568
:1055E0005095609570958091DB039091DC03A091BC
:1055F000DD03B091DE038A019B01082319232A23CE
:105600003B23C901B8011F910F910C944E2A0F93AF
:105610001F9341E050E060E070E004C0440F551F6C
:10562000661F771F8A95D2F78091DB039091DC0388
:10563000A091DD03B091DE038A019B0108271927A1
:105640002A273B27C901B8011F910F910C944E2ABC
:105650000F931F930091DB031091DC032091DD0376
:105660003091DE03602B712B822B932B1F910F91B6
:105670000C944E2A0F931F930091DB031091DC03CF
:105680002091DD033091DE03602371238223932375
:105690001F910F910C944E2A0F931F930091DB03DF
:1056A0001091DC032091DD033091DE036027712728
:1056B000822793271F910F910C944E2A08958F9261
:1056C0009F92AF92BF92DF92EF92FF920F931F9340
:1056D000CF93DF9300D000D01F92CDB7DEB76B839E
:1056E0007C838D838A018C819D81892B31F01F3FC2
:1056F00031F481E04F3F19F403C081E001C080E044
:1057000080FF03C080E090E04DC08B818823D1F101
:105710008090DB039090DC03A090DD03B090DE036B
:105720008091DF039091E003A091E103B091E20347
:10573000882A992AAA2ABB2A8FE1E82EF12CD501C2
:10574000C4010E2C04C0B695A795979587950A9429
:10575000D2F780FD06C081E0E81AF10880F7D12C6D
:1057600007C0DE2CB8018E2D0E94900C019799F392
:1057700080E1189FF0011124E55AFC4FE00FF11D64
:10578000D08209C080E1189FF0011124E55AFC4F36
:10579000E00FF11DD08009831A8369817A818D2DF4
:1057A0000E94900C0F900F900F900F900F90DF9130
:1057B000CF911F910F91FF90EF90DF90BF90AF902E
:1057C0009F908F90089590911101992379F1909174
:1057D0001201992359F1982F9695969596959F3198
:1057E000A1F0E0911301F0911401E90FF11D877010
:1057F00021E030E0A90102C0440F551F8A95E2F76D
:10580000CA019181892B818308959091060490FFAC
:1058100029C01F928F9388EF97E09F938F930E94E8
:105820004F050F900F900F900F9008952091130146
:1058300030911401F90132969FEF40E051918517A4
:1058400089F09F3F19F4511101C0942F4F5F4E31E1
:10585000A9F79F3F39F0F901E90FF11D97FDFA957E
:1058600082830895089590911101992381F1909177
:105870001201992361F1982F9695969596959F31EF
:10588000A9F0E0911301F0911401E90FF11D877067
:1058900021E030E0A90102C0440F551F8A95E2F7CC
:1058A000CA0180959181892381830895909106048E
:1058B00090FF1CC01F928F938AED97E09F938F9368
:1058C0000E944F050F900F900F900F900895E09158
:1058D0001301F09114019F01225E3F4F92818913C1
:1058E00001C012823196E217F307C1F7089581E0F3
:1058F00090E0E0911301F0911401E80FF91F10827C
:10590000019680329105A9F70895809105040895C4
:1059100090910504892B80930504089580959091BA
:105920000504892380930504089580930504089550
:1059300010920504089590910404892B8093040427
:105940000895809590910404892380930404089518
:105950001092040408958093E30308951092E303E2
:1059600008958091130190911401FC0131969C01DE
:10597000205E3F4F80E0919191118F5FE217F30716
:10598000D1F70895E0911301F0911401809105047D
:105990008083E0911301F0911401908180910404BF
:1059A000892B80838091E303882361F0E0911301C8
:1059B000F09114019081892B80830E94B12C811178
:1059C0001092E30380911301909114010C94E61F4F
:1059D00090937F0180937E0108958295982F937311
:1059E00044E0949F900111248C7C86958695282B09
:1059F000822F8575880F2A7A2695822B0895CF935A
:105A0000DF93D92F0E94ED2CC82F8D2F0E94ED2CF3
:105A10002C2F30E0322F2227A901482BCA01DF9119
:105A2000CF91089508950895CF93DF9300D000D0CB
:105A30001F92CDB7DEB70F900F900F900F900F9081
:105A4000DF91CF910895089508950C94532180E03B
:105A5000089583B7817F8C6083BF83B7816083BFE4
:105A60007894889583B78E7F83BF0895CF930E94E3
:105A70009D210E9407170E949E21C0E08C2F0E944A
:105A8000850C892B29F4CF5FC830C1F780E001C0B5
:105A900081E0CF9108950E948E0C0C94EC221F920D
:105AA0000F920FB60F9211248F939F93AF93BF93D2
:105AB0008091070490910804A0910904B0910A0410
:105AC0004196A11DB11D8093070490930804A093F3
:105AD0000904B0930A04BF91AF919F918F910F90E9
:105AE0000FBE0F901F90189582E084BD93E095BD86
:105AF0009AEF97BD80936E0008952FB7F894809128
:105B0000070490910804A0910904B0910A042FBFE2
:105B100008952FB7F894609107047091080480915C
:105B2000090490910A042FBF08959C014FB7F8947F
:105B30008091070490910804A0910904B0910A048F
:105B40004FBF821B930B089578941F920F920FB64C
:105B50000F9211248F939F93AF93BF93809107046B
:105B600090910804A0910904B0910A040196A11D26
:105B7000B11D8093070490930804A0930904B09387
:105B80000A04BF91AF919F918F910F900FBE0F901C
:105B90001F9018950E946A1EF89487E797E79093E4
:105BA00001088093000887E090EBDC0180932104DA
:105BB00090932204A0932304B09324049CE088E1F2
:105BC0000FB6F894A895809360000FBE9093600084
:105BD000FFCF80E090E00895089580910D0480FF4C
:105BE0000BC06091180185E0689FB0011124759584
:105BF0006795759567952BC081FF09C06091180165
:105C000085E0689FB00111247595679520C082FFDB
:105C100007C06091180185E0689FB001112417C08A
:105C200090910E049923D1F060911701961788F78F
:105C30002091180185E0289F90011124929FA001D6
:105C4000939F500D112470E0CA010E94CB3160383F
:105C5000710540F46115710519F406C065E070E046
:105C6000862F08958FE7089581E0089580910D04AF
:105C700080FF08C06091160170E075956795759575
:105C8000679521C081FF06C06091160170E075958F
:105C9000679519C082FF04C06091160170E010C0C2
:105CA00090910E04992399F0609115019617A0F731
:105CB00080911601899FC001112470E00E94CB31B0
:105CC0006038710540F46115710519F406C061E092
:105CD00070E0862F08958FE7089581E00895803F52
:105CE00021F40E94ED2D819504C0813F29F40E948A
:105CF000ED2D809311040895823F21F40E94ED2D33
:105D0000819504C0833F29F40E94ED2D80931004F7
:105D10000895893F19F40E94362E05C08A3F31F458
:105D20000E94362E81958093120408958B3F21F4B2
:105D30000E94362E819504C08C3F29F40E94362E95
:105D4000809313040895843F21F480910F048160AF
:105D500017C0853F21F480910F04826011C0863FF7
:105D600021F480910F0484600BC0873F21F480915F
:105D70000F04886005C0883F31F480910F04806172
:105D800080930F0408958D3F21F480910D0481606C
:105D90000BC08E3F21F480910D04826005C08F3FBF
:105DA00029F480910D04846080930D040895803F50
:105DB00039F48091110487FF6CC01092110469C0FE
:105DC000813F29F4809111041816BCF362C09091B0
:105DD0001004823F29F497FF5CC01092100459C050
:105DE000833F19F41916CCF354C0893F41F48091D4
:105DF000120418160CF04DC0109212044AC08A3FCB
:105E000029F48091120487FF44C0F6CF8B3F39F408
:105E10008091130487FF3DC0109213043AC08C3F59
:105E200029F4809113041816BCF333C0843F21F485
:105E300080910F048E7F17C0853F21F480910F045D
:105E40008D7F11C0863F21F480910F048B7F0BC0A2
:105E5000873F21F480910F04877F05C0883F31F48C
:105E600080910F048F7E80930F0413C08D3F21F427
:105E700080910D048E7F0BC08E3F21F480910D0424
:105E80008D7F05C08F3F29F480910D048B7F809317
:105E90000D048091100481110EC0809111048111B4
:105EA0000AC080911204811106C0809113048111EF
:105EB00002C010920E0408958091060483FF7EC0F4
:105EC0008DE398E00E94B60480910F041F928F9397
:105ED00088E398E09F938F930E944F0586E398E0B4
:105EE0000E94B60480911004282F082E000C330B5A
:105EF0003F938F9383E398E09F938F930E944F0586
:105F000081E398E00E94B60480911104282F082EA6
:105F1000000C330B3F938F938EE298E09F938F9307
:105F20000E944F058CE298E00E94B6048091120412
:105F3000282F082E000C330B3F938F9389E298E0B3
:105F40009F938F930E944F0587E298E00E94B604CA
:105F500080911304282F082E000C330B3F938F934E
:105F600084E298E09F938F930E944F0581E298E02E
:105F70000E94B60480910E041F928F938EE198E0E8
:105F80009F938F930E944F058CE198E00E94B60486
:105F900080910D041F928F9389E198E09F938F93D6
:105FA0000E944F0586E198E00E94B6048DB79EB727
:105FB0004C960FB6F8949EBF0FBE8DBF8FE094E055
:105FC0000E942F200E947D2D90930C0480930B043F
:105FD00008951F93CF93DF9380910B0490910C044D
:105FE0000E94952DAC0190910E04992321F02091EF
:105FF000190130E006C020911A018AE0289F900123
:1060000011244217530708F485C080911004C091F1
:106010001104D091120410911304811107C0C11111
:1060200075C0D11173C0111171C074C09F3F19F0B8
:106030009F5F90930E04181624F40E94ED2D809318
:1060400010048091100487FF05C00E94ED2D8195FA
:10605000809310041C1624F40E94ED2D80931104EB
:106060008091110487FF05C00E94ED2D81958093DA
:10607000110460911004662331F1C0911104CC2306
:1060800011F1062E000C770B880B990B0E94D23071
:1060900023E333E343E35FE30E9436310E949A3007
:1060A000609310046C2FCC0F770B880B990B0E9418
:1060B000D23023E333E343E35FE30E9436310E94AF
:1060C0009A30609311041D1624F40E94362E80939A
:1060D00012048091120487FF05C00E94362E81951C
:1060E00080931204111624F40E94362E8093130418
:1060F0008091130487FF05C00E94362E81958093FE
:106100001304DF91CF911F910C945C2F9F3F09F0F6
:106110008FCFA0CFDF91CF911F910895EFE0F4E0F2
:1061200085E0DF011D928A95E9F710920E04109226
:106130000D0408950E94A1306894B1110C9430317F
:1061400008950E94153188F09F5798F0B92F99272C
:10615000B751B0F0E1F0660F771F881F991F1AF052
:10616000BA95C9F714C0B13091F00E942F31B1E057
:1061700008950C942F31672F782F8827B85F39F056
:10618000B93FCCF3869577956795B395D9F73EF4EB
:1061900090958095709561957F4F8F4F9F4F089593
:1061A000E89409C097FB3EF49095809570956195B1
:1061B0007F4F8F4F9F4F9923A9F0F92F96E9BB2767
:1061C0009395F695879577956795B795F111F8CFE3
:1061D000FAF4BB0F11F460FF1BC06F5F7F4F8F4F4E
:1061E0009F4F16C0882311F096E911C0772321F044
:1061F0009EE8872F762F05C0662371F096E8862FDC
:1062000070E060E02AF09A95660F771F881FDAF732
:10621000880F9695879597F9089557FD9058440FE4
:10622000551F59F05F3F71F04795880F97FB991FF5
:1062300061F09F3F79F087950895121613061406B2
:10624000551FF2CF4695F1DF08C01616170618063F
:10625000991FF1CF86957105610508940895E8941A
:10626000BB2766277727CB0197F908950E9449310C
:106270000C94BA310E94AC3138F00E94B33120F056
:10628000952311F00C94A3310C94A93111240C9492
:1062900030310E940D3170F3959FC1F3950F50E09E
:1062A000551F629FF001729FBB27F00DB11D639FC8
:1062B000AA27F00DB11DAA1F649F6627B00DA11D6E
:1062C000661F829F2227B00DA11D621F739FB00D14
:1062D000A11D621F839FA00D611D221F749F332784
:1062E000A00D611D231F849F600D211D822F762F1D
:1062F0006A2F11249F5750409AF0F1F088234AF0FA
:10630000EE0FFF1FBB1F661F771F881F9150504065
:10631000A9F79E3F510580F00C94A3310C943031C5
:106320005F3FE4F3983ED4F3869577956795B795EC
:10633000F795E7959F5FC1F7FE2B880F911D969506
:10634000879597F9089597F99F6780E870E060E076
:1063500008959FEF80EC089500240A9416161706FE
:1063600018060906089500240A9412161306140646
:1063700005060895092E0394000C11F4882352F0A9
:10638000BB0F40F4BF2B11F460FF04C06F5F7F4F61
:106390008F4F9F4F089597FB072E16F4009407D058
:1063A00077FD09D00E94E83107FC05D03EF49095B6
:1063B00081959F4F0895709561957F4F0895EE0FD9
:1063C000FF1F0024001C0BBE0790F691E02D0994DE
:1063D000AA1BBB1B51E107C0AA1FBB1FA617B7070B
:1063E00010F0A61BB70B881F991F5A95A9F7809527
:0C63F0009095BC01CD010895F894FFCFFA
:1063FC0005EA010000FF3317D517A6176A173617E1
:10640C00010101E4032808140A321E5F5A313530A9
:10641C00005F3F3F3F3F005F415438340041540020
:10642C005854005445524D494E414C004E4F4E4528
:10643C00004D4F55534500494E54454C4C49004C6A
:10644C004F474954454348004558504C4F524552CC
:10645C000044454641554C5400397F224407C5063B
:0E646C00A3064F066806810600100008000413
:106800008800EA44E944E244040005000600070069
:10681000080009000A000B000C000D000E000F001C
:1068200010001100120013001400150016001700CC
:10683000180019001A001B001C001D001E001F007C
:10684000200021002200230024002500260027002C
:10685000280029002A002B002C002D002E002F00DC
:10686000300031003200330034003500360037008C
:10687000380039003A003B003C003D003E003F003C
:1068800040004100420043004400450046004700EC
:10689000480049004A004B004C004D004E004F009C
:1068A000500051005200530054005500560057004C
:1068B000580059005A005B005C005D005E005F00FC
:1068C0006000610062006300640065A185006700EC
:1068D000680069006A006B006C006D006E006F005C
:1068E0007000710072007300890087008A008B00BD
:1068F000E000E100E200E300E400E500E600E7007C
:106900000100010001000100EA4401000100E2442D
:106910000100010001000100460001004A004B0097
:10692000010001004700480001000100E9440100A6
:106930000100010001000100010001003A003B00DC
:106940003C003D003E003F0040004100420043004B
:10695000010035004C0039000100440045005200A0
:1069600049000100010050004F0029004D004E0079
:1069700051000100010001000100010001000100BF
:1069800001000100010001000100010001000100FF
:1069900001000100010001000100010001004D00A3
:1069A0004A004E004B0001000100010001000100FF
:1069B00001000100010001000100010001000100CF
:1069C00001000100010001000100010001000100BF
:1069D00001000100010001000100010001000100AF
:1069E0000100010001000100490001000100010057
:1069F000010001000100010001000100010001008F
:00000001FF
